:10000000831603308500860183129C019D019F01A8
:10001000A82882070434013402340234043404343E
:10002000023401340234013404340234043402341E
:10003000013404340434013401340434023401340E
:1000400002340134043402340434023402340134FE
:1000500004340234043402340134043404340134EA
:100060000134043402340134FF34FF348601860342
:100070005E20E73086005E20C33086005E2081303F
:1000800086005E2086015E20813086005E20C330BF
:1000900086005E20E73086005E20860186035E20B3
:1000A000860108000A3090005E20900B542808005A
:1000B000033090005E20900B5A28080064309B00AB
:1000C00000009A0B602805181F149B0B602808007D
:1000D0000E0886005E2086015E200E0886005820ED
:1000E000860158200E0886005220522052205220AD
:1000F000860152209C0A9D0A9D0A080004309E0039
:1001000086015E205E2086035E205E209E0B802896
:100110008601080004309E008601860A860D0318B9
:1001200093285E208E28860C5E20860C031C942863
:100130009E0B8C288601080004309E00F03086005B
:1001400058200F30860058209E0B9E2886010800FC
:1001500036201F1CA8281C0809209100911FB228D6
:100160009C01AB28111CB6287E20BB28911CBA2804
:100170008A20BB289C2052201D0809209200921F33
:10018000C3289D01BB28121CC92833308E0068206B
:10019000AB28921CCF2873308E006820AB286D30BE
:0601A0008E006820AB2870
:00000001FF
